:100000008A110A120528000009000730990083169A
:100010000510851005118512051685158312E83027
:10002000A0000330A1001C23AF01A721B401851D4E
:100030001A2853201F3083056430A000A1011C231F
:100040003208013EB200051E2628E7201F30830536
:1000500032080A3C031D3028B2013308013EB300C8
:100060001F30830533083C3C031D3A28B301340894
:10007000013EB4001F30830534080F3C03184F289D
:100080002F08003C031D4628A7214A281F3083055E
:100090007B21AF011F308305B401B301B2011F30D2
:1000A00083051728522885140130AF00B0010130B4
:1000B000B100B201B301B4013108013C031DCF28E6
:1000C000B101AC012C08323C031C7028851D6A2844
:1000D0000130B1001F3083050130AC07031C6228DA
:1000E0001F3083056430A000A1011C233208013EAB
:1000F000B20032080A3C031D8128B2013308013ED8
:10010000B3001F30830533083C3C031D8B28B3012B
:100110003408013EB4001F308305AC012C08323C8A
:10012000031C9C28851D96280130B1001F308305D3
:100130000130AC07031C8E281F3083053008003CBB
:10014000031DAE283408033C031DAC28CE218510C6
:100150000130B000B401B3011F3083051F308305A7
:10016000AC012C08323C031CBF28851DB928013086
:10017000B1001F3083050130AC07031CB1281F30CC
:1001800083053408063C031DCC287B2185140A23F3
:100190008510B401B301B2011F3083055C281F3004
:1001A00083052C30A0000130A1001C233308003C43
:1001B0000318DB28FF211F3083053230A000A10186
:1001C0001C2385100E30B4002D30B3000800051537
:1001D0000130AF00B0010130B100B201B301B40190
:1001E0003108013C031D6329B101AC012C08323CEC
:1001F000031C0429051EFE280130B1001F308305B1
:100200000130AC07031CF6281F3083056430A000C2
:10021000A1011C233208013EB20032080A3C031837
:100220001529B2013308013EB3001F30830533089E
:100230003C3C031D1F29B3013408013EB4001F30AC
:100240008305AC012C08323C031C3029051E2A29E9
:100250000130B1001F3083050130AC07031C222997
:100260001F3083053008003C031D42293408033C3D
:10027000031D4029DE2105110130B000B401B30196
:100280001F3083051F308305AC012C08323C031C52
:100290005329051E4D290130B1001F30830501305F
:1002A000AC07031C45291F3083053408063C031D99
:1002B00060297B2105150A230511B401B301B201A0
:1002C0001F308305F0281F3083052C30A00001303B
:1002D000A1001C233308003C03186F29FF211F30A5
:1002E00083053230A000A1011C2305110E30B4009B
:1002F0002D30B30008008514F430A0000130A100B7
:100300001C231B22C4223E22C4227222C422FF21AB
:10031000C4220122C422F621D2228510F430A0008A
:100320000130A1001C230515F430A0000130A1000C
:100330001C231B22C4223E22C4227222C422FF217B
:10034000C4220122C422F621D222051108008514FC
:10035000F430A0000130A1001C231B22C4223E2245
:10036000C4227222C422FF21C4220122C422F62107
:10037000D22285100515F430A0000130A1001C2305
:100380001B22C4223E22C4227222C422FF21C42284
:100390000122C422F621D222051108008514F4306E
:1003A000A0000130A1001C232F22C4223422C42229
:1003B0003C22D2220A23C422851008000515F430FD
:1003C000A0000130A1001C232F22C4223422C42209
:1003D0003C22D2220A23C42205110800E822F92275
:1003E0000800F922E822E822E8220800F922E8229F
:1003F000F922E8220800F922E822E8220800E8228F
:100400000800E822E822F922E8220800F922F9226D
:10041000E8220800E822E822E822E8220800E82290
:10042000E8220800E822F922F922F9220800F9223C
:10043000E822F9220800E822F922E822E82208004E
:10044000F922F9220800F922E8220800F922F9220B
:10045000F9220800E822F922F922E8220800F9220C
:10046000F922E822F9220800E822F922E82208000D
:10047000E822E822E8220800F9220800E822E8221F
:10048000F9220800E822E822E822F9220800E822FE
:10049000F922F9220800F922E822E822F9220800CC
:1004A000F922E822F922F9220800F922F922E822A9
:1004B000E8220800F922F922F922F922F92208009B
:1004C000E822F922F922F922F9220800E822E8229A
:1004D000F922F922F9220800E822E822E822F9228A
:1004E000F9220800E822E822E822E822F92208009E
:1004F000E822E822E822E822E8220800F922E8229D
:10050000E822E822E8220800F922F922E822E8227B
:10051000E8220800F922F922F922E822E82208005C
:10052000F922F922F922F922E8220800E822F92228
:10053000E822F922E822F9220800F922F922E82229
:10054000E822F922F9220800E822E822F922F92219
:10055000E822E8220800F922E822E822F922E8222B
:100560000800F922E822E822E822F9220800F9220C
:10057000E822E822E822E822F92208008512463023
:10058000A000A1011C23080085124630A000A10193
:100590001C234630A000A1011C234630A000A1016D
:1005A0001C23080085124630A000A1011C23463000
:1005B000A000A1011C234630A000A1011C2346304D
:1005C000A000A1011C234630A000A1011C230800AB
:1005D0008516053084000130AA007030A00002307A
:1005E000A1003830A2000030A30057238512BE229C
:1005F00008008516053084000130AA007030A00084
:100600000230A100E030A2000030A3005723851281
:10061000BE2208008516053084000130AA00703023
:10062000A0000230A100B030A2000430A300572384
:100630008512BE2208001B2BA0080319272B2E238E
:10064000A003000000000000000000001C2BA10817
:10065000031908002E23A103A0031C2B0C30A500B6
:10066000A50B302B000000001230A200A20B3D2B86
:100670003F233F230000000008003F23362B0D30AE
:10068000A400A40B412B000008001030A8020001B8
:10069000031C013EA902031C08004E2B0A30A802CD
:1006A0000001031C013EA902031C08004E2B2A086E
:1006B00080042008A8002108A90045230130A202D7
:1006C000031CA3032A0980052008A8002108A9000B
:1006D0004523A208031D572BA308031D572B080011
:02400E00C431BB
:00000001FF
